:020000020000FC
:1000000017C018951895FDC018951895189518954E
:100010001895189518951895189518951895010222
:100020000400000040404000000001010100000009
:1000300022240FE50DBF02E00EBF00E806BD00E080
:1000400006BD379843E0A0E6BB27EEE1F0E002C032
:1000500005910D93E033E1F7BFD013D002E076D0E5
:1000600034E604D0332702D001D0FDCF12D011D016
:1000700010D00FD00ED00DD034D033D027D026D012
:100080000895EEE8F0E0332751E00ED008954040A7
:10009000400054E0ECE9F0E007D008952A2A2A5500
:1000A00055552A2A2A555555C6E60591099304E661
:1000B00026D0332339F4759079928590899204E69D
:1000C0001ED001C053D05A9579F7089554E0E6ED5B
:1000D000F0E0EADF08952A5555552A2A2A55555544
:1000E0002A2A54E0ECEEF0E0DFDF08952A2A555585
:1000F000552A2A2A5555552A1197F1F708950F9335
:10010000BF93AF93B3E1A8E8F7DF0A95D9F7AF91B2
:10011000BF910F910895A32FBB275096AF93BF9324
:10012000B2E0AFEDE9DFBF91AF911197B9F7089554
:100130000F93AF93BF930F930AE0E1DFE9F70F91BD
:100140000A95C9F7BF91AF910F9108950F93CF937F
:10015000DF93CAE00F9304E6D2DFCA95E1F70F916F
:100160000A95B9F7DF91CF910F9108955F93599058
:10017000688075908590AA24082D162D27D00095AB
:100180000395C02EAA0C072D152D20D0B02E0C0DD6
:10019000502F219759926882BEDF571004C0681013
:1001A00002C05F910895952E990C9C1434F05C0D5B
:1001B000A0FC02C0539401C05A94B91454F35B0DCF
:1001C000A1FC02C06394E5CF6A94E3CF011B18F44D
:1001D000A394009503950895F89403E0332427B37E
:1001E000E0E6FF271191212B0A95E1F727BB20BEFE
:1001F00028E020BF20E429BF2FBC2FEF2EBD78942C
:1002000008950F930FB70F932F931F93EF93FF93BF
:100210004423C9F0413031F14230E1F13394032DF0
:10022000033009F43324ECE6E30D0081002331F0C0
:1002300028B3E0E6E30D0081022B08BB2FBC1EE3D0
:100240001EBD44272BC0E6E6E30D10811EBD41E034
:100250002FBC1EB5121103C01FEF1FBD1FC010E43D
:1002600018BF1CC0ECE6E30D2081222339F028B32F
:10027000E0E6E30D00810095022308BBE6E6E30D0E
:1002800000811FEB42E00E3B08F043E0101B1EBD57
:100290002FBC04C043E02FBC0FEF0EBDFF91EF91C8
:0C02A0001F912F910F910FBF0F91189527
:00000001FF
